:020000040000FA
:060000000BEF18F01200E6
:0600080004EF08F01200F5
:060018000CEF08F01200DD
:061000000BEF18F01200D6
:0610080026EF16F01200B5
:0610180028EF16F01200A3
:06102A0003006E3000001F
:1010300099000000050000006C3000009E000000D8
:101040000200000064300000F80200000800000008
:10105000F9EC0CF06A6A686A9F0E6B6EFB0E696EA3
:101060006D8C6D9C6E6AD4EC0CF0DF6ADF500B6EF9
:101070000C6A100E0B5C000E0C5810E2DF50040DD1
:10108000F3CFE9FFF4CFEAFF000EE926040EEA22CF
:10109000EE6AEE6AEE6AEE6ADF2AE8D7160E706E26
:1010A00068A604D0030E9EEC0CF0FAD70201DE6BAA
:1010B000E36BE46BE56B6D98080ED26F040ED36F93
:1010C000C46BC36BFCEF0CF0F9EC0CF00201C351E4
:1010D0000BE16D6A696A6DB602D06D86FCD70201BC
:1010E000010EC36F160E6F6EC30508E16DBA06D010
:1010F000686A696A69806988020EC36F6850040B68
:1011000004E06950040B01E065D86DB249D0685025
:10111000010B11E06950010B0EE09ADF0201040E91
:10112000C36F0401400E026F040E036F080E016FBF
:10113000006B8C0E00136850100B04E06950100B0C
:1011400001E042D86850400B08E06950400B05E0D0
:1011500095EC16F0060E9EEC0CF06850200B04E0A7
:101160006950200B01E01ED86850020B06E0695060
:10117000020B03E096EC16F06A6A040E0201C35DEE
:101180000FE369A60DD0DF6A040EDF5C09E268A6F2
:1011900007D06CCFEBF2030ED1DB26D8DF2AF4D7D1
:1011A000FCEF0CF070A00DD0C5EC0CF0EF508008F7
:1011B00007E1CEDBEF50840803E1E7DB8C0EEF6E36
:1011C0007090050E9EEF0CF06984040EB7DB6D8203
:1011D00093EF16F06D9294EC16F0699468A403D026
:1011E000020EACDBFBD71200FD0E0201EB1519E17C
:1011F0007E0EEB15E8407F0B040DF3CFC6F2F4CF63
:10120000C7F2000EC627040EC723C6C2C8F2C7C263
:10121000C9F2C87565EC0DF002E117EF09F028EF8F
:1012200009F0FD0EEB15040801E11AD8120090DB5D
:10123000EF50800B02E08CDBEF6A0201DA6BDB6BB4
:10124000DF6BE06BDE6B96D897EC16F0E6EF0AF0FA
:10125000020E0201DB5D02E170EF0BF05CEF09F0C2
:10126000C8DB76DBEF50400B01E0010EDF6E0201C0
:10127000D275080EC35D09E142C46EFF6E500008CE
:1012800002E2100E01D0040EC36FDB0513E157EC30
:101290000DF0D4D9020E0201DA5D03E159DB840EB0
:1012A00007D0DF5003E154DBC80E02D051DB880EBB
:1012B000EF6E01D001D8A0D352EC0DF0030EE12661
:1012C000020E0201DB5D2CE16D50100B29E05DDBAD
:1012D000EE52EF500B6E0C6A080E0B1821E10C5009
:1012E0001FE165EC0DF01CE1BEDBEF50800B18E157
:1012F000BADBCCDBDF6ADF500B6E0C6A080E0B5CCE
:10130000000E0C5822E2DF507FDBDF50EA6A400F0C
:10131000E96E040EEA22E552E750EF6EDF2AEBD7C2
:10132000DB6BBADBEF6A040ED2190B6ED3C20CF082
:10133000010E0BC0DBFF020ED3C2DBFF010EDBCFC1
:10134000E9FF020EDBCFEAFFEF6A0201E3AF0CD048
:10135000E651E71107E005D0E7C2FAFF0201E651C6
:10136000F96EFADF0201E39F030EE15C02E2E16A3B
:10137000E552FCD204014051600BE842E842E842E9
:10138000E842E842000901E0120041510C0A43E042
:101390000B0A3FE00C0A31E0010A22E00B0A1EE0D2
:1013A000020A1CE0030A18E0080A10E0010A0CE037
:1013B0000F0A08E0030A01E012000201DE8F080EA6
:1013C000C36F120072EF0AF0C9EF0BF00201C40EF6
:1013D000DC6F020EDD6F0CD0ADEF0AF00CEF0AF0FF
:1013E00044510201DC6FDD6BC50EDC27020EDD23EC
:1013F000DE81010EDF6FDE8F12000201DE8F04013D
:101400004451EA6AC50FE96E020EEA2242C4EFFFB8
:10141000120099EF16F0120045DB050EE1260401DB
:10142000420510E140511F0B00090CE10201DE8F63
:10143000030E0401415D04E10201010EEA6F02D0D6
:101440000201EA6B0401425147E140511F0B0208BF
:1014500043E144510F0B00093FE00201DE8F040E0F
:10146000DB6A020EF36E040EDBCFF4FFF350F45C84
:1014700033E2F4DA040EDBCFE6FF04014451800BC3
:1014800001E0010EC9DAE552E724A5DA030E415D59
:1014900003E163DA840E1CD044510F0B0C6A700F09
:1014A0000B6E0F0E0C22020E0BC0DBFF030E0CC0E6
:1014B000DBFF020EDBCFE9FF030EDBCFEAFFEE908E
:1014C000ED5244AF03D049DA400E02D046DAC80EDE
:1014D000EF6E040EDB2AC5D7050EE15C02E2E16A7D
:1014E000E55244D2800E0401405D36E10201C00E97
:1014F000DE6F04014351030A1EE0010A09E0030AFA
:1015000029E10201490EDC6F2E0EDD6F120E1FD095
:101510009ADA0E0EF6262F0E87DA020E0201F76A0D
:10152000DC25F66EDD51F7220900F5CFDFF20A0067
:10153000F5CFE0F2120087DA100EF6262F0E74DADD
:10154000DCC2F6FFDDC2F7FF0800F5500201DF6FD5
:10155000E06B12000201DE6B120004DA0401486B3A
:10156000496B40511F0B020A11E0030A0CE0010A0B
:101570001DE10201DE8F040148810201EA0516E146
:101580000401488313D00201DE8F10D00201DE8FE8
:1015900065DA04014451800B01E0010E3DDA1BDAEB
:1015A000DCD9EF50040B02E0010E486F0201DEAF00
:1015B00007D0480EDC6F040EDD6FDE81020EDF6F98
:1015C000020EE15C02E2E16AE552D0D16D980201BF
:1015D000DEBF07D0E3AF02D093DA28D05DDA840E05
:1015E00026D0E3BF2AD0040140AF23D00201DF514F
:1015F0000401465D0201E0510401475904E246C47A
:10160000DFF247C4E0F21AD80201010EDB6F8FD976
:10161000B6D9800EEF6EB9D9EE52080EEF6EB5D97D
:1016200035DAB3D9800EEF6E42DA92D9C80EEF6E7A
:101630001200020165DAC80EEF6E120093D90201A2
:10164000080EDF5D000EE0590DE2DFC2DEFFE0C2F2
:10165000DDFFDA5102E1010E03D0DA0506E1020EE8
:10166000DA6F03D0080EDE6EDD6A72D9EF9270D9A0
:10167000EF906ED9010EDB50EF126AD9EE52DFCF38
:10168000EFFF000EDB50DF5F010EDB50E05B480E2A
:10169000E86F040EE96FDEB10FD0DCD91BE0DCC2CD
:1016A000F6FFDDC2F7FFDC2B000EDD230800F5504E
:1016B00084D9F3E2DB06F1D7CDD90CE0DCC2E9FF37
:1016C000DDC2EAFFDC2B000EDD23EF5076D9F4E219
:1016D000DB06F2D7020EE15C02E2E16AE55246D196
:1016E00041D953D9EE52EFCFDFFFDFCF0BF00B50D4
:1016F0000201E45D000EE55903E2E4C2DFFF09D018
:10170000DF500B6E0C6AE850E45DE46F0C50E55955
:10171000E56F010EDB6ADF50F36E010EDBCFF4FFE5
:10172000F350F45C10E2010EDB506ED9E1C2E9FF28
:10173000E2C2EAFFE12B000EE223E552E750EF6E32
:10174000010EDB2AE8D7000ED880E455000EE555DF
:101750000CE2CAD91AD9EF50400B03E184D9C80E64
:1017600002D081D9880EEF6E0ED07DD98FD9E65187
:10177000E71107E005D0E7C2FAFF0201E651F96E72
:10178000FADF0201E39F020EE15C02E2E16AE55248
:10179000EDD00201DE8F08D9010EE66EE66AE66A38
:1017A000C50EE66E020E98D942C4C4F2040142513D
:1017B00004E10201100EC36F12000201200EC36F7C
:1017C0009AEF16F0CFD84AD9E5D8040DF3500B6E36
:1017D0000C6A020E0F0B05E0D8900C320B32E806B3
:1017E000FBE1D8900B360C36D8900B360C367FD9EF
:1017F0000B50EE260C50ED22B0D8EF9EFD0EDB50C4
:1018000002E159D901D05CD9EA22DECFEEFFDDCF6B
:10181000EDFFA3D8EF9CA1D8040EE926000EEA2222
:10182000EF8C020EE15C02E2E16AE5529FD09AD8A9
:10183000FE0EDB500C6A700F0B6E0F0EDFD8FD0E24
:10184000DB50E66E8AD8E552E750EE6EED6AFD0E8B
:10185000DBA402D0E66AF0D8FD0EDBA203D0010EB5
:10186000E66EEAD8020EE15C02E2E16AE5527ED061
:1018700079D8FE0EDB5004E10FD9840EEF6E05D04F
:1018800089D8F6D887D8010FF3D8020EE15C02E2BE
:10189000E16AE5526BD066D8FD0EDB5002E010D94C
:1018A00001D009D9EA22EECFDEFFEDCFDDFF55D81A
:1018B00032D9FB0EDBCFEEFFFC0EDBCFEDFF4DD8B8
:1018C000EE52FA0EDBCFEFFF400E47D8E850EF168E
:1018D000880E43D8E850EF12FD0EDB5002E0F0D83E
:1018E00001D0E9D8EA22EF74DECF0BF0DDCF0CF0A7
:1018F0000BC0F3FF0CC0F4FF020EE15C02E2E16AF0
:10190000E55234D0CFD8010EF36EFC0EDB5004E06C
:10191000D890F336E806FCE1F31C0B6EFD0EDBCF2E
:10192000E9FFFE0EDBCFEAFF0B50EF16E5D09BD8A8
:10193000EE52080EEF6E97D88BEF0DF0E66E680E44
:10194000E66E0F0EE66EDEDFE552E552E55212005E
:10195000D2C2E9FFD3C2EAFF1200DECFE9FFDDCF3A
:10196000EAFF12009FD8020EE1261200E16EC4D0F9
:10197000FE0EEA6ADB34FE0BEA36E96E1200400E18
:10198000EE6E040EED6E33EF0DF0C6C2E9FFC7C276
:10199000EAFF1200FD0EDB50E8240D6EFE0EDB5058
:1019A000040DF3500D241200020EE66EE66AE66A9C
:1019B000710EE66E0F0E6CEF0DF0E66EE8C2E9FFF9
:1019C000E9C2EAFFE82B000EE923E552E750EF6E8B
:1019D000DF06010E1200040DF4CF0CF088D8F3508E
:1019E000EE260C50ED221200480EEE6E040EED6E47
:1019F000120058D8E6521200E5527ED00C220BC0DD
:101A0000DEFF0CC0DDFF1200EA6A480FE96E040E2B
:101A1000EA22EF50E66E1200E8240D6E44510F0BDF
:101A2000040DF3500D241200F7220900F5CFDCF26B
:101A30000A00F5CFDDF21200FE0EDBCFE6FFC2DEBC
:101A4000E552E55212004251F66EF76AD890F6362A
:101A5000F73612004CD8EE50ED101200000EDE6E7C
:101A6000040EDD6E1200C8C2E9FFC9C2EAFF12000F
:101A7000040DF3CF0BF0F4CF0CF0000E0B26040E88
:101A8000BDDF840E6ADFE850EF12120044D8400E2A
:101A9000EE6E040EED6E12004ADF71DF8C0EEF6EFB
:101AA000A8EF0CF0D9CFE6FFE1CFD9FF120050DF4D
:101AB00032D8F4EF0CF05CDFCA0EE926020E1200F9
:101AC00057DFD20EE926020E12005FDFEF503C0B0B
:101AD000E842E8420D081200E66EDAEC17F00B6EF1
:101AE000050EE15E0B50120022DFF4EF0CF0D9CFAF
:101AF000E9FFDACFEAFF1200E552E7CFD9FF120083
:101B0000020EDB6F25DFEE52EF6A22DFC80EEF6EAA
:101B1000EBDF33EF0DF0020EE926000EEA22120091
:101B2000400EE66E000EE66E020EE66EC9EC14F094
:101B3000E552E552E55200090CE060C085F0020173
:101B4000F95103E085C0E6FF08D085C0E6FF4FDA13
:101B500005D00201F95104E0E66AABD9E552120062
:101B6000F95112E18B50800B0FE1FDC20BF0FEC268
:101B70000CF0FD07000EFE5B0B500C1005E1E66853
:101B800019EC18F0E55215D81200936831DB4CDBE4
:101B9000D6DA4ADB899848DB89868984DBDADADAA7
:101BA0008B9ED8DAD7DAD6DAD5DA0201FD69FE697A
:101BB0001200899889968994899A9368C0DA8B8EE5
:101BC0001200BFDAE652FE0EDB50DF6EDF98DF9ABE
:101BD000DF9CDF9EFE0EDB90DB92DB94DB96DB3836
:101BE0000F0BE76EFE0EE7CFDBFFDB5004DBF5CF1C
:101BF0007FF0DF5000DBF5CF80F0E552A7D293688D
:101C00008984898689988BDA8998898698DA936A93
:101C10008A6A95DA84DA200E8A6E91DA80DA8FDAAF
:101C2000936889888CDA8150120079DA8150120029
:101C300088DA89848986899882DA936A8A6A6FDA6F
:101C4000FE0EDB508A6E6BDA936889887FD279DA70
:101C5000E652DF6A8150DF6E62DADF50E55276D2FB
:101C6000560E0201005D10E1560E015D0DE100010E
:101C7000615111E10001780E626F2D0E636F00015A
:101C8000030E81DA010E06D00001615104E164DA2D
:101C9000010E79DA616F0201F96B120052DA02016A
:101CA000F95105E100C27AF0010EF96F08D000C2C7
:101CB0007BF0F96B7AC000F27BC001F2D1DF46D233
:101CC00040DA83DA2EE10001795170DA01E673DA45
:101CD00018E3DF6ADF506ADA01E66DDA02E2BCDAA5
:101CE000F9D70201FA5104E00001792B0201FA6BE5
:101CF0000001615102E137DA4BDA0001795111E15B
:101D00000DD079517F080DE3DF6A010EDB50DF5CF7
:101D100002E2A2DAFAD727DA60DA8B8E0201100E1D
:101D2000F96F020EE15C02E2E16AE552E16E0ED269
:101D300008DA4BDA2DE10001795138DA01E63BDAB5
:101D400018E3DF6ADF5032DA01E635DA02E28FDAD1
:101D5000F9D70201FA5104E00001792B0201FA6B74
:101D60000001615102E1FFD913DA0001795110E15C
:101D70000CD079517F080CE3DF6A010EDB50DF5C89
:101D800002E275DAFAD7EFD928DA0201100EF96FFC
:101D9000020EE15C02E2E16AE552E16ED7D1D1D9EF
:101DA000030EE126020EDB6A520E02010125022516
:101DB0000325E76E020EE7CFDBFFDB50045D0AE090
:101DC0000001615104E1C8D9010EDDD9616F020142
:101DD000F96B24D002C2DFFF010E03C2DBFF01C298
:101DE00079F00001795104E179690201010EFA6F7D
:101DF000DF501F0806E30201FB6B030EF96F98DF4B
:101E00000DD0010EDBCFE6FFDFCFE6FF11DFE5529D
:101E1000E5520201FB6B040EF96F52DF030EE15C29
:101E200002E2E16AE552E16E91D106DAFE0EDB5084
:101E3000DF5C16E2010EDBCFF3FFDB2AF350EA6A28
:101E4000000FE96E020EEA22EF50E66E0201F85131
:101E5000F82BEA6A7A0FE96E000EB2D9DF2AE6D7CC
:101E6000020EE15C02E2E16AE552E16E6FD1E4D973
:101E7000FE0EDB50DF5C14E2010EDB50EA6A7A0FE3
:101E8000E96E000EEA22EF50E66E010EDB50EA6AC0
:101E9000000FE96E020E94D9010EDB2ADF2AE8D783
:101EA0000201F86B020EE15C02E2E16AE552E16ECA
:101EB0004DD147D9E6520201F951100A01E187D00C
:101EC000180A73E00F0A45E0010A3DE0030A28E022
:101ED000010A21E0070A1AE0010A0CE0030A05E002
:101EE0000001615101E07FD07CD0FE0EDBCFE6FF28
:101EF000D5DE59D0050EF85D02E374D901D082D940
:101F0000050E0201F85D71E36DD96FD000016151DA
:101F10006CE10EDF6AD00001615167E1D1DE65D06E
:101F2000FF0E0001915D09E10201F96B9AC040F2D8
:101F3000000161515AE11DD958D0912B0001926BDB
:101F400043EC13F052D0FE0EDBCFE6FFA8EC11F00D
:101F50002AD0FE0EDB5012E1FF2B640EE66EF4EC8D
:101F600017F0E5520201FF5140E1000161513BE1F0
:101F7000140EE66E2E0E53D9E55235D0410E0201F5
:101F8000005D0AE10201080EF96F000161512DE1C7
:101F90007E0EE66E2D0E06D00001615126E1140E74
:101FA000E66E2E0E3CD9E55220D0A96AAA0EA86E84
:101FB000A69EA69CA684550EA76EAA0EA76EA68204
:101FC000050EE66E19EC18F0E552A6940CD000014F
:101FD00061510BE1FCC240F2CCD80201F96BFC6B01
:101FE00004D031D9616F0201F96BE552AFD0A9D8A5
:101FF000E652DF6A02010051390A01E184D0010A88
:1020000001E17FD00F0A6DE0010A68E0030A5BE09E
:10201000010A56E0070A51E0010A41E0030A3BE0E9
:10202000700A2DE0310A01E178D0200A76E0030A37
:1020300074E0240A72E02F0A70E00F0A19E0250A02
:102040006CE0200A0BE0040A04E00001615165E144
:1020500062D0020EDDD861E303DE5FD096DD040EB0
:10206000D7D802E39CDE59D0CDD80201020E11D0A0
:102070008CDDFE0EDBCFE6FF3CEC11F04AD0000118
:10208000615105E1E00EE66E2D0EC9D8E552020160
:10209000070EF96F42D0B3DD81D83FE103D0C5DD33
:1020A0007DD83BE100017F0E626F000E636F00017F
:1020B000020E666F0001010E21D0F2EC12F02DD05D
:1020C00036EC13F02AD00201050EF96F0001200E44
:1020D000916F0001926B43EC13F01FD015EC13F0DD
:1020E0001CD084EC13F0899881CF00F1000161517C
:1020F00014E139D80001010E666F0001676F00011D
:102100000BD076D802D090D8899A010EE66E19ECE1
:1021100018F0E55202D097D8616FE55217D084D8F5
:10212000899482D8898414EF11F080D8EA22EF5084
:102130000201FC25FC6F00017907DF2A12000A0E5C
:1021400091D0D9CFE6FFE1CFD9FF1200E552E7CF1A
:10215000D9FF1200FE0E86D000017B0E626F2D0E9D
:10216000636F000112000001000E626F010E636FC9
:1021700012000001400E626F020E636F0001010E3B
:10218000666F000165D0666F0001676B0001120089
:102190000001800E666F0001010E5AD0DF6EDFCFA6
:1021A000E6FF0FDDE5520001615112000B6E0C6A73
:1021B000D8900C501200800E0B5C000E0C581200D0
:1021C000EA22E552E750EF6E1200020EE126010E00
:1021D00079C0DBFF000161511200010EDBCF66F018
:1021E000000136D0050EE66E42DEE552CFEF0EF06E
:1021F0001BD8898A1200F76A670FF66E2D0EF72238
:1022000008001200FE0EDBCFE6FF0FDEE5521200E3
:10221000F36EFE0EDBCFF4FFF350F45C1200E66EBB
:1022200034EC15F0E5521200010E1CD0DF50EA6AC2
:10223000000FE96E010E120084DF020EE126010E8E
:10224000DB6ADF6A120088DF020E9DDF010E1200DA
:10225000676F0001616F1200FADCE66EE7DFB0DF46
:1022600095EF10F0E66E19EC18F0E5521200DEDF83
:08227000EA22EF6895EF10F07F
:0822780094DA030EE1260201D5
:10228000FC6B0201FA6B040EF36EFE0EDBCFF4FF63
:10229000F350F45C56E30201060EF96F01C279F0C7
:1022A00002C291F003C292F00001795104E1796910
:1022B0000201010EFA6F570E0201012502250325C6
:1022C0000201FC6F0001915101E1D0D9200E000103
:1022D000915D0DE290510BE0C80EE66EF4EC17F044
:1022E000E55212DABCD8FF0802E10001906B200E23
:1022F0000001915D01E199D9040EDF6EFE0EDB5005
:10230000DF5C15E2DF506DDA010EEFCFDBFF200E50
:102310000001915D06E3010EDBCFE6FF7AD8E552BE
:1023200002D0010EDB50E76E020E4FDAE7D7020152
:10233000FA5105E0020E00017925796F02D0000103
:10234000792B030EE15C02E2E16AE552E16E2ED2E6
:1023500028DA060EE126030EDB6AFE0EDB500001D2
:10236000795D0CE1FE0EDB06DB503BDA020EEFCFAF
:10237000DBFF010EF36E030EF3CFDBFFDF6AFE0E11
:10238000DB50DF5C15E2DF502CDA040EEFCFDBFF11
:10239000200E0001915D06E3040EDBCFE6FF39D885
:1023A000E55202D0040EDB50E76E050E0EDAE7D7D9
:1023B000030EDB5014E0020EDB500201FC5D0FE166
:1023C00016DA02E100019B6B000161511BE1000183
:1023D0005E0E626F300E21DA0001616F13D0030EC2
:1023E000DB5010E0020EDB500201FC5D0BE0FCC292
:1023F00040F20001615102E1E1D916DAF8D902E1B7
:1024000000019B6B060EE15C02E2E16AE552E16EBF
:10241000CDD1C7D9FE0EDB50FF080AE100019B5168
:1024200007E0898618DA07DA12DAFE0EDB5016D0DA
:10243000AFD9A00E06DAFE0EDBCFE6FF92C0E6FFB4
:1024400091C0E6FF96D8E552E552E5520001010E33
:102450009B6FFE0EDBCFE6FF65D8E552A7D1D9CF43
:10246000E6FFE1CFD9FFE6529368010EE66E19EC64
:1024700018F0E5528988010EE66E19EC18F0E55265
:102480000000000000008150DF6E010EE66E19ECC6
:1024900018F0E5528998010EE66E19EC18F0E55235
:1024A000DF5000D0E552E552E7CFD9FF120079D9CD
:1024B000FE0EDB50800BE76EFE0EE7CFDBFFCBD9C5
:1024C0008150800B04E0FE0EDB50800806E0815056
:1024D000800B06E1FE0EDB5003E1B9D9010E02D0FC
:1024E000B6D9000E63D19368B6D981AA02D0AFD90C
:1024F000010CADD9000C55D9E652ADD9A00E81140E
:10250000DF6EFE0EDB50A00BE76EFE0EE7CFDBFFAB
:10251000DB50DF5C03E19BD9010E02D098D9000E9D
:10252000E55244D13ED9E652936800019A6BDF6AC6
:10253000080EDF5C19E263D913E168D911E1D3DF3A
:10254000000910E05CD90EE161D90AE10001010E39
:102550009A6F81CF40F2FE0EDBCF41F2F00E2AD906
:102560007EDF05D0DF2AE4D70001020E9A6FE55224
:102570001DD117D900019B5105E18998898689846D
:1025800085D905D08986898856D98998936A67D96B
:1025900093680CD106D98998899689844CD90F0EF5
:1025A00068D974D95CD98986936800D1FAD8E65283
:1025B0000F0EC16E926A93689492898A899889866F
:1025C000898470D9E2D837D9FE0EDB508A6EDDD807
:1025D00032D9DBD840D993688150DF6E38D9DF50CB
:1025E000E552E4D0DED8E652D3D8900E2AD9E66A76
:1025F000200EE66EDBDFE552E552DF6EDFCF40F204
:10260000010EE66EE66AD2DFE552E552DF6EDFCFFD
:1026100041F2F00ECFD80001615105E12FD9000140
:10262000616F0201F96BE552C1D06ED818DFFF0867
:1026300008E059DF010808E1E6685DDFE5520108BE
:1026400014E10001906B1200E66855DFE5520009C5
:102650000CE105DF0201406F0001615102E1AED8DB
:10266000E3D8F00EA7D80201F96B1200899890D830
:10267000800EE7D88DD8300E9DD80001010E906FE6
:10268000FE0E39EF14F08DD8020EE126DF6A010E3E
:10269000DB6ADB500B6E0C6AD8900C5004E6FF0E20
:1026A0000B5C000E0C580CE2DFCFE6FFB2DEE55209
:1026B000050EDFD8DF2A0001922B010EDB2AE9D7B5
:1026C000FF0E0001915D02E100019B6B00019A0584
:1026D00014E19A6B0001615102E1D0D80CD0020ED6
:1026E00000019A5D0AE10001615107E10001560E07
:1026F000626F300E92D80001616F020EE15C02E25F
:10270000E16AE552E16E52D0898489968998010E7A
:10271000E66E19EC18F0E5528994010EE66E19EC9C
:1027200018F0E5528984010EE66E19EC18F0E552B6
:1027300089988996936A010E8A6E010EE66E19ECED
:1027400018F0E5528994010EE66E19EC18F0E55286
:102750008984010EE66E19EC18F0E552200E8A6E9F
:102760000000010EE66E19EC18F0E5528994010E96
:10277000E66E19EC18F0E5528984010EE66E19EC4C
:1027800018F0E552000093681200010E39EF14F0C2
:10279000AA0E57D8550EE66EAA0EE66E020EE66E2B
:1027A00074D0D9CFE6FFE1CFD9FF1200E552E7CFD1
:1027B000D9FF1200E66EE66AE66A67D00001400EB5
:1027C000626F020E636F00011200E7CFDBFF0001B2
:1027D000922BDB500201FC25FC6F00017907DF2AF8
:1027E0001200EA6A000FE96E020EEA2212000201EC
:1027F000F96B0201FC6BFF0E0001915D1200FE0EF1
:10280000DBCFE6FF54DEE55200091200FE0EDBCFFF
:10281000E6FF71DEE55200091200636F0001010E50
:10282000666F0001676B1200010E666F0001676F33
:102830000001616F1200A9DF8994A7DF8984C5EFC9
:1028400013F0E66E550EE66E050EE66E26D09DDFA1
:102850008998C5EF13F099DF8988C5EF13F095DFEC
:10286000899A93DFFC0EDB508A6E8FDF898AC5EF71
:1028700013F0E66E19EC18F0E55212009FDF020E1D
:10288000666F0001010E676F120007D00BD8D3DF0F
:10289000FE0EDB508A6E1BEF14F07CDEE552E55233
:1028A000E5521200936AFD0EDB508A6E1BEF14F0A6
:1028B000040140511F0B010801E012004051600B60
:1028C000E842E842E842E842E842010801E012003A
:1028D000445103E0440501E012004151220A31E075
:1028E000030A24E0010A15E0210A0DE0010A01E0D3
:1028F00012000201710EDC6F000EDD6F080EDF6F3B
:10290000E06BDE8121D00201710EDC6F000EDD6F05
:102910001BD046C4E4F247C4E5F20201D80EE16FD1
:10292000040EE26FE66BE76BE38F12000201D80E34
:10293000DC6F040EDD6F070EDF6FE06BC10EDE6F24
:10294000120042C46CF00201DE8F12000401D86B49
:10295000C20ED96F010EDA6FDB6BDC6BDD6B080E1C
:10296000DE6F0001616B606B1A0EE66E020EE66EA2
:1029700017EC0CF0E552E5521E0EE66E030EE66E05
:1029800017EC0CF0E552E55246D900016A6B6B6B0F
:1029900012002CD90001606B6851691102E1000E30
:1029A00005D034D9EF50800B01E0010E00092DE174
:1029B000FC0EDBCF0BF02AD9EE52EF50D8800B542F
:1029C00005E224D9EE52FC0EEFCFDBFF606BFC0E6C
:1029D000DB50605D19E26051EA6A580FE96E040E3F
:1029E000EA22EF50E66E6051E76EFD0EDBCFE9FFA5
:1029F000FE0EDBCFEAFFE750E926000EEA22E552A1
:102A0000E750EF6E602BE3D706D900016051F3D099
:102A1000EDD80001615107E1E2D8FC0EDBCF66F092
:102A2000010E676F616FE7D00BD917E1BDD8E7D80A
:102A300002E10C500BE0010EDBCFE9FFDB2A020EB6
:102A4000DBCFEAFF01E3DB2AEF50F1E1C8D8DFCFAB
:102A500066F00001010E676F616F030EE15C02E238
:102A6000E16AE552E16EC7D0EBD818E19DD8C7D82E
:102A700002E10C500CE0010EDBCFF6FFDB2A020E68
:102A8000DBCFF7FF01E3DB2A0800F550F0E1A7D820
:102A9000DFCF66F00001676B010E616F030EE15C32
:102AA00002E2E16AE552E16EA6D0A0D8020EE1266C
:102AB00000016A516B1102E1000E08D06AC0E9FF03
:102AC0006BC0EAFFEF50800B01E0010E00095CE1F2
:102AD000030E615D01E1616B615156E0020E615DC3
:102AE00008E1E66A000EE66EE66AA2D80001030E6F
:102AF00043D0610542E1400E0B6E0C6A66510B5CDF
:102B0000000E0C5803E2400EDF6E02D066C0DFFFFD
:102B1000DF50665D666F980E646F040E656F010E80
:102B2000DFCFDBFF67510BE1010EDB5012E062C02B
:102B3000F6FF63C0F7FF0800F55044D8F5D7010E43
:102B4000DB5007E062C0E9FF63C0EAFFEF503AD80C
:102B5000F6D70001665111E16AC0E9FF6BC0EAFFD8
:102B6000EE52EF500B6E0C6A400E0B1804E10C5045
:102B700002E1020E01D0030E616FDFCFE6FF980E77
:102B8000E66E040EE66E54D8020EE15C02E2E16AE3
:102B9000E552E16E30D0030EE66E4BEC0CF00B6E9E
:102BA000050EE15E0B501200DF6AFD0EDBCF06F072
:102BB000FE0EDBCF07F0DE5206C0DEFF07C0DDFFF2
:102BC000DD52120064C0E9FF65C0EAFFEF6E642BBE
:102BD000000E6523622B6323010EDB061200FD0E3F
:102BE000DBCF62F0FE0EDBCF63F01200D9CFE6FF41
:102BF000E1CFD9FF1200E552E7CFD9FF1200DF2A5B
:102C0000DF500B6E0C6AFF0E0B18120068C0E9FF54
:102C100069C0EAFF1200400EE66E580EE66E040E22
:102C2000E66EE66AB8DFF3CF68F0F4CF69F0120021
:102C3000010EE66EB0DFF3CF6AF0F4CF6BF0120056
:0C2C4000D5DF030EE126000161511200F7
:042C4C0083D8110018
:102C5000D8CFE4FFE0CFE4FFE46E7CD8E550E5CFC9
:102C6000E0FFE5CFD8FF100008D864EC08F090EC46
:102C70000DF022D855EC15F0F8D70F0EC16E070EE7
:102C8000B46EF26A28EC08F046EF16F08B8E936A69
:102C9000816A926A946A806A826A8B9E9484949014
:102CA0008B80949E929892969294929A8998899603
:102CB0008984898A8B9E120004D8200E0201C35D8C
:102CC000120000019E519F1104E1100E9E6F270E0D
:102CD0009F6F9E07000E9F5B6DA204D09E519F11B7
:102CE00021E116D00201C3510AE0C30503E0020E40
:102CF000C35D02E18B801200040EC35D02E18B9084
:102D00001200100EC35D06E100019E519F110AE101
:102D10008B701200200EC35D05E100019E519F11D2
:102D200001E18B701200120012001200120058EF25
:102D300014F01200A6EF14F06D840201080EC16FAA
:102D4000070EC26FC107000EC25BC151C211FAE18A
:102D50006D941200DACFE4FFE652E552E5CFDAFFD8
:022D600012005F
:0E2D62001B5B324A003031323334353637389D
:102D70003941424344454600011E323F3F000D0A9F
:102D80002050757474696E67206465766963652088
:102D9000696E746F20626F6F74206C6F616465720E
:102DA000206D6F64652E205265706C7567206465B8
:102DB0007669636520616E642075736520484944B7
:102DC00020626F6F746C6F6164657220746F206C29
:102DD0006F6164206669726D77617265200D0A000B
:102DE0001B5B324A200D0A2050726573732041200C
:102DF000616761696E20746F20636F6E6669726DC2
:102E000020626F6F746C6F61646572206D6F6465B2
:102E1000200D0A000D0A20426F6F746C6F616465AB
:102E200072206D6F64652063616E63656C6C6564B0
:102E30002E2046726F6D2075736572206F7220743C
:092E4000696D6F7574200D0A0024
:072E4900120100020200006B
:102E500008D8040A0001000102000109024300022F
:102E60000100C03209040000010202010005240033
:102E700010010424020205240600010524010001BA
:102E80000705820308000209040100020A0000008D
:102E90000705030240000007058302400000040309
:102EA000090434034D006900630072006F00630081
:102EB000680069007000200054006500630068002D
:102EC0006E006F006C006F00670079002000490001
:102ED0006E0063002E0038034300440043002000CE
:102EE000520053002D003200330032002000450014
:102EF0004500430020004A003300200050007200CB
:102F00006F006700720061006D00650072005B2E4B
:062F10009E2EA22ED62E1B
:0A2F16002A0EF66E100EF76E000E84
:102F2000F86E00010900F5508B6F0900F5508C6FA9
:102F300003E18B6701D03DD00900F550866F090091
:102F4000F550876F0900F550886F09000900F550AA
:102F5000E96E0900F550EA6E090009000900F55014
:102F6000896F0900F5508A6F09000900F6CF8DF0CE
:102F7000F7CF8EF0F8CF8FF086C0F6FF87C0F7FF4F
:102F800088C0F8FF0001895302E18A5307E0090075
:102F9000F550EE6E8907F8E28A07F9D78DC0F6FF83
:102FA0008EC0F7FF8FC0F8FF00018B07000E8C5B0F
:042FB000BFD7120075
:0C2FB400FE0EE3CFE9FFFF0EE3CFEAFFC3
:102FC000E9CFF3FFEACFF4FFFB0EE35003E1FC0E81
:102FD000E35009E0FB0EE30602E2FC0EE306FD0E01
:082FE000E350EE6EF1D7120080
:082FE800FF0EE3500F6EEF0E27
:102FF00001D0F30EE76EE72EFBEF17F00C0E0E6E0E
:10300000E76AE72E01EF18F00E2E00EF18F00F2EF2
:06301000F9EF17F01200B9
:0A30160013EE00F023EE00F0F86A5C
:103020000A9C8BEC17F031EC18F034EC16F0FBD75F
:0230300012008C
:0E303200FF0EE350E84E1200000000D000D068
:0830400000D0E82EFAD71200BF
:0830480000EE00F00F0EEE6A2D
:06305000EA62FDD7120048
:0830560074696D656F7574006B
:02305E004F0021
:0230600021004D
:0230620012005A
:08306400000000000000000064
:02306C00000062
:02306E00000060
:033070000000005D
:020000040030CA
:0100000024DB
:010001000EF0
:0100020039C4
:010003001EDE
:010005008179
:010006008178
:010008000FE8
:01000900C036
:01000A000FE6
:01000B00E014
:01000C000FE4
:01000D0040B2
:00000001FF
